:04000000A0016428CF
:100008000800102080040C281020FF3A80050D28D5
:10001800FF3A841780055F2894000630941905304C
:10002800840000308A00140807398207013402343A
:100038000434083410342034403480348F018E0066
:100048006400FF308E07031C8F07031C0800033071
:100058008D00DC30312024288D01E83E8C008D098C
:10006800031C3B28FC308C07031837288C078D0F9E
:1000780036288C183F288C1841280C18432808006B
:100088008D018F018E0054200239031DFF305F2837
:100098008D018F018E0054200139031DFF305F2828
:1000A8000F080D02031D5C280E080C020319023408
:1000B800031C0434013483130313831264000800FF
:1000C80005308400083009200530840004300920F8
:1000D80005308400023006200530840001300920F4
:1000E8000630840010300920063084004030092092
:1000F8000630840080300920063084002030092032
:100108006400861C88288428063084001030062065
:10011800053084000830062013308F0088302320F3
:100128000530840004300620063084004030062064
:10013800A601A701A801A9010130A800A901280862
:100148008C0029088D008F0132304E20031DC128F4
:100158000130A600A70126088C0027088D00FD3075
:100168008F00E8304E20031DBD28A60A0319A70AF0
:10017800AF28A80A0319A90AA32805308400023069
:100188000920063084008030062090308B008B17C1
:10019800D0288B1B0800252907308F00D03023205A
:1001A800CD200530840001300620CD2006308400A3
:1001B80020300620CD206400061DEE28CD206400E6
:1001C800061C2529CD208B17EC288B1B0800252918
:1001D800DF28E9200530840002300620E9200630B7
:1001E800840080300920E920C8302220E920053029
:1001F800840001300920E9200630840020300920DD
:10020800E92007308F00D0302320E9200530840012
:1002180004300920E9200630840040300920E92014
:1002280075308F0030302320E920053084000830F5
:100238000920E9200630840010300920E9208428AC
:10024800E9200530840002300620E92006308400C9
:1002580080300920E92001308F00F4302320E92084
:100268000530840001300920E92006308400203060
:100278000920E92001308F00F4302320E9206400B0
:10028800861DC128E9206400061DEE28E9204329BF
:02029800E9205B
:084000007F007F007F007F00BC
:04400E00F53F010079
:00000001FF
